:020000040000FA
:10000000840A77001402F50177031102F2017703E5
:10001000030477030E02EF0177030B02EC01770371
:100020000802E90177031702FF0F26000400000809
:100030001802C10178037803F80100087B007C00F6
:100040000109A802E802E8000109AB02EB02EB009B
:100050000109AE02EE02EE000109B102F102F10067
:100060000109B402F402F4000109FC02340A010996
:10007000FB02200A00087B00010908028A00010C2B
:100080000307FF0C4306000CE80101090B028D0079
:10009000010C0307FF0C4306000CEB0101090E02E3
:1000A0009000010C0307FF0C4306000CEE01010950
:1000B00011029300010C0307FF0C4306000CF10131
:1000C000010914029600010C0307FF0C4306000C03
:1000D000F40101091A023C000000000000000000C9
:1000E0000000000001090000000000000000000006
:1000F000FC02720A0000010900000000000000007C
:100100000000FB023C0A0008000C06009F0C0200E5
:10011000D40A180918023F0E3900100CF901180909
:1001200018021F0E3A00040CFA01010C3D001809D8
:1001300018027F0E2A00400CEA01180918027F0EEF
:100140002D00400CED01180918027F0E3000400C04
:10015000F001180918027F0E3300400CF301180952
:1001600018027F0E3600400CF6011D076A003D079D
:100170006D005D0770007D0773009D0776003B09E9
:100180003B093B09180918021F0E3E001D021F0FF4
:100190007E014306C20A1E023D00F902970A1E09AB
:1001A0001E091E09D20A880A000C2B00000C2E0022
:1001B000000C3100000C3400000C2D00000C30004D
:1001C000000C3300000C3600020C3A00B00C2A0080
:1001D0003B09060C3A003B09020C3A00300C2A009D
:1001E0003B09040C3A003B09020C3A00FF0C2A00C0
:1001F0003B09060C3A003B09020C3A00300C2A007D
:100200003B09040C3A003B09020C3A00FF0C2A009F
:100210003B09060C3A003B09200C3A00100C2A005E
:100220003B09030C3A003B09050C3A00000C2A007C
:100230003B09010C3A003B0966071F0BD40A000C6E
:100240002800000C2A00FF0C2D00F00C3A003B099E
:10025000FF0C2B00FF0C2D00FF0C3000FF0C3300B7
:10026000FF0C3600400C3A003B09100C3D00000C1E
:100270003100000C3300000C3400000C3600030C7D
:100280003A003B09FF0C3100FF0C3300FF0C340037
:10029000FF0C3600010C3A003B09FD02370B000C45
:1002A0003000000C3300000C3600100C2A00300C1B
:1002B0003A003B091D022D003F0C2D011D023000AC
:1002C0001E0233001D0236001E02F601010C3A0028
:1002D0003B093B09250CFD01290CFE0166075A0B61
:1002E000FF0C3000FF0C3300FF0C3600400C3A00CE
:1002F0003B09120C3D00000C3100000C3300000CD7
:100300003400000C3600020C3A003B09FF0C3100AF
:10031000FF0C3300FF0C3400FF0C3600010C3A00D8
:100320003B09FD027B0B000C2D00000C3000000C83
:100330003300000C3600100C2A00C00C3A003B09B8
:100340003B09D40AF00C2800800C2B00400C2E0036
:10035000200C3100100C3400A3041E09A305A304D3
:02036000880A09
:021FFE00EE0FE4
:00000001FF
